:020000040000FA
:100000008316851086100610061583128F019C0139
:100010009C14861006148510861402304720861022
:10002000103084000C308E00000006108001061D88
:1000300080140000840A0614000000008E0B1528AE
:100040001008980011089000911099109A109B10B8
:100050000F3084000E308E000508FD3900040418AE
:10006000023A8500840A4E30472000008E0B2C286F
:100070008510FF304720FF304720FF304720FF30FA
:1000800047204F3047200000000064000C288C00FF
:060090008C0B482808005B
:02400E00FE3F73
:00000001FF
